:100000000C94CE040C9406050C9406050C9406057D
:100010000C9406050C9406050C9406050C94060534
:100020000C9406050C9406050C9480240C9452251F
:100030000C94BF1E0C9406050C9406050C94060542
:100040000C9406050C9406050C9406050C94060504
:100050000C9406050C94471F0C9406050C94060599
:100060000C9406050C9406050C9406050C940605E4
:100070000C9406050C9406050C9406050C940605D4
:100080000C9406050C9406050C9406050C940605C4
:100090000C9406050C9406050C9406050C940605B4
:1000A0000C9406050C9406050C940605C908C908AD
:1000B000F508F5085D09880A880A880A7B09140A88
:1000C000250A250A091BF71A101B661ABD1BBD1B42
:1000D000F41ABD1BBD1B3D1BBD1B511B9D1BBD1B36
:1000E000BD1BBD1BBD1B711BBD1BBD1B6E1BBD1BEB
:1000F000291BBD1BBD1BB71BB71BB71BB71BB71BF2
:10010000B71BB71BB71BB71BB91BBD1B091BEC1AD1
:10011000BD1BBD1BBD1BBD1BBD1BBD1BBD1BBD1B1F
:10012000BD1BBD1BB91BBD1BBD1BF41ABD1BB51BE5
:10013000B51BB51BB51BB51BB51BB51BB51BB51B3F
:10014000B91BBF25E625DE26E625DE263226552606
:10015000DE26AC26BB2629002B002A0067005300B0
:100160005400550056005F006000610057005C00BD
:100170005D005E00000059005A005B0058006200FC
:1001800000006341000029002B002A006700530093
:100190005400550056005F0060006100005C5C0088
:1001A0005D005E00000059005A005B0058006200CC
:1001B00000006341000044454255473A206469739A
:1001C00061626C65642E0A0044454255473A2065D9
:1001D0006E61626C65642E0A000A00253032580098
:1001E0006C65645F7461736B3A20004F6E65736871
:1001F0006F743A206163746976653A2025640A0059
:100200000A0025303862003A200025303258000AB2
:10021000722F632030313233343536370A00626151
:10022000636B6C6967687420737465703A20257518
:100230000A006261636B6C6967687420646973614A
:10024000626C650A006261636B6C69676874206543
:100250006E61626C650A006261636B6C69676874E9
:1002600020746F67676C653A2025750A00626163C8
:100270006B6C696768742064656372656173653A65
:100280002025750A006261636B6C69676874206978
:100290006E6372656173653A2025750A003F0043FD
:1002A0003E20004C25640A000A092D205374617415
:1002B0007573202D0A686F73745F6B6579626F6167
:1002C00072645F6C65647328293A20253032580ABD
:1002D0006B6579626F6172645F70726F746F636F68
:1002E0006C3A20253032580A6B6579626F6172640E
:1002F0005F69646C653A20253032580A6B65796D08
:1003000061705F636F6E6669672E6E6B726F3A2005
:10031000253032580A74696D65725F7265616433A5
:100320003228293A202530386C580A000A092D2035
:1003300056657273696F6E202D0A5649443A203013
:10034000784645454428414D4A29205049443A20A1
:100350003078363036302850414429205645523ABC
:10036000203078303030330A4255494C443A20200E
:10037000284665622032372032303232290A4F5007
:1003800054494F4E533A204C5546412045585452FB
:10039000414B455920434F4E534F4C4520434F4D01
:1003A0004D414E44204E4B524F20343039360A478F
:1003B00043433A20352E342E30204156522D4C499D
:1003C00042433A20322E302E30204156525F415265
:1003D00043483A20617672350A000A092D20436F9E
:1003E0006E736F6C65202D0A4553432F713A097166
:1003F0007569740A000A092D204D61676963202D13
:100400000A443A094465627567204D6573736167F4
:100410006520546F67676C650A583A094D617472BC
:100420006978204465627567204D6F646520546F5C
:1004300067676C65202D2053686F77206B65797036
:1004400072657373657320696E206D61747269786B
:1004500020677269640A4B3A094B6579626F617271
:100460006420446562756720546F67676C65202D52
:100470002053686F77206B65797072657373207293
:1004800065706F72740A4D3A094465627567204D54
:100490006F75736520546F67676C650A563A095625
:1004A000657273696F6E0A533A0953746174757398
:1004B0000A433A09416374697661746520436F6E3B
:1004C000736F6C65204D6F64650A46312D4631307F
:1004D0003A0953776974636820746F204C617965B9
:1004E0007220302D392028463130203D204C3029D3
:1004F0000A302D393A0953776974636820746F2084
:100500004C6179657220302D390A47524156453A7F
:100510000953776974636820746F204C6179657240
:1005200020302028616C7465726E617465290A42FE
:100530003A094A756D7020746F20426F6F746C6F4A
:10054000616465720A4553433A094A756D702074B7
:100550006F20426F6F746C6F616465722028616CEC
:100560007465726E617465290A453A095072696E44
:100570007420454550524F4D2053657474696E6721
:10058000730A4253504143453A09436C65617220F6
:10059000454550524F4D0A4E3A094E4B524F20544A
:1005A0006F67676C650A006261636B6C696768748A
:1005B0005F636F6E6669672E7261773A202530320D
:1005C000580A2E656E61626C653A2025750A2E6C9C
:1005D0006576656C3A2025750A006B65796D6170EA
:1005E0005F636F6E6669672E7261773A20253032DD
:1005F000580A2E737761705F636F6E74726F6C5FF1
:10060000636170736C6F636B3A2025750A2E6361AA
:1006100070736C6F636B5F746F5F636F6E74726F18
:100620006C3A2025750A2E737761705F6C63746C69
:100630005F6C6775693A2025750A2E737761705F64
:100640007263746C5F726775693A2025750A2E7340
:100650007761705F6C616C745F6C6775693A2025B7
:10066000750A2E737761705F72616C745F72677563
:10067000693A2025750A2E6E6F5F6775693A2025E5
:10068000750A2E737761705F67726176655F657357
:10069000633A2025750A2E737761705F6261636B20
:1006A000736C6173685F6261636B73706163653AF9
:1006B0002025750A2E6E6B726F3A2025750A00642C
:1006C000656275675F636F6E6669672E7261773A00
:1006D00020253032580A2E656E61626C653A2025FD
:1006E000750A2E6D61747269783A2025750A2E6B31
:1006F0006579626F6172643A2025750A2E6D6F7597
:1007000073653A2025750A006565636F6E666967D3
:100710003A0A64656661756C745F6C617965723AFA
:100720002025750A003F004E4B524F3A206F6666F7
:100730000A004E4B524F3A206F6E0A000A6D6F75D9
:1007400073653A206F66660A000A6D6F7573653AC5
:10075000206F6E0A000A6B6579626F6172643A20DD
:100760006F66660A000A6B6579626F6172643A208F
:100770006F6E0A000A6D61747269783A206F66665E
:100780000A000A6D61747269783A206F6E0A000A75
:1007900064656275673A206F66660A000A6465627E
:1007A00075673A206F6E0A000A0A4A756D70696EA5
:1007B0006720746F20626F6F746C6F616465722E56
:1007C0002E2E2000433E2000436C656172696E67E7
:1007D00020454550524F4D0A000A0025303258201E
:1007E000006B6579626F6172645F7265706F7274BD
:1007F0003A200064656C5F6B65795F6269743A20CA
:1008000063616E27742064656C3A20253032580A83
:10081000006164645F6B65795F6269743A2063614B
:100820006E2774206164643A20253032580A005BD8
:10083000735D005B575D005B535D005B525D005B69
:10084000445D005B435D000803500041004400002C
:1008500000080341004D004A000000040309040998
:10086000025B00030100A0FA09040000010301017A
:100870000009211101000122400007058103080041
:100880000109040100010300000009211101000118
:10089000226D000705820320000109040200020303
:1008A0000000000921110100012222000705830335
:1008B00020000107050303200001120100020000CF
:1008C0000008EDFE60600300010200010631FF092F
:1008D00074A1010975150026FF0095207508810295
:1008E0000976150026FF00952075089102C00501C4
:1008F0000980A101850319012AB700150126B70057
:10090000950175108100C0050C0901A1018504192C
:10091000012AA002150126A002950175108100C0D0
:1009200005010906A1018506050719E029E715005B
:1009300025019508750181020507190029EF1500A9
:10094000250195F075018102050819012905950514
:1009500075019102950175039101C005010906A178
:1009600001050719E029E7150025019508750181A2
:10097000029501750881010507190029FF15002658
:10098000FF009506750881000508190129059505E0
:1009900075019102950175039101C00011241FBEDC
:1009A000CFEFDAE0DEBFCDBF04B603FE18C0809102
:1009B0008A0290918B02A0918C02B0918D028730B7
:1009C000904BA740B04B59F410928A0210928B02C0
:1009D00010928C0210928D02E0E0F8E3099511E08C
:1009E000A0E0B1E0E8EAFFE402C005900D92AC3867
:1009F000B107D9F722E0ACE8B1E001C01D92AA38F6
:100A0000B207E1F70E948F160C94D2270C940000D5
:100A1000FF93EF93E0918C01F0918D01309709F0F5
:100A20000995EF91FF910895FC018591803011F0B7
:100A3000EFDFFBCF0895FF27E0E230E247FF0CC075
:100A4000419597FF09C0EDE260957095809590956E
:100A5000611D711D811D911D27FF02C0219530E38D
:100A600050E2AA27660F771F881F991FAA1FA41795
:100A700010F0A41B63955A95A9F7AA3008F0A95F56
:100A8000A05DAF93F395611571058105910541F75F
:100A9000ED3211F4EF93F395F21718F43F93F395B9
:100AA000FBCF8F91B5DFFA95E1F70895E991F991C0
:100AB0008591803021F0853219F0AADFF9CF0895B1
:100AC00020E0E89455915532C1F3503311F4689405
:100AD00055915A3348F4505390F3220F022E220FAF
:100AE000220F200D250FF4CF0EF4219589919991B5
:100AF000533619F3533729F1533559F1BC0188277F
:100B00009927E8945C3621F48991999168945591DC
:100B1000543639F446EF7EF077FF0DC08FEF9FEF2C
:100B20000AC055374AE039F0583540E121F05236D5
:100B300042E009F00895FF93EF937DDFEF91FF917D
:100B4000B7CFFF93EF93FC0181918030B9F360DF61
:100B5000FBCFFF93EF9368DFF1CFDF93CF93CDB758
:100B6000DEB72596A3DFCF91DF91089581E0089548
:100B700081E008950C94B80508950C94BC051F936A
:100B8000CF93DF9300D000D01F92CDB7DEB749835B
:100B90005A836B8330918F0189819A81311114C0FE
:100BA000662359F0222349F00E94BF0C182F682FAA
:100BB00089819A810E946A0C03C00E94940C182FAC
:100BC00069817A81812F04C00E94BF0C69817A817A
:100BD0000F900F900F900F900F90DF91CF911F917A
:100BE0000C94E213FC01262F4081518162817381B4
:100BF00084810C94BF0581E00895CF93DF93EC01CD
:100C000060E00E94F205BE01DF91CF910C94BD051A
:100C10000C9452150C944E1508950E94140B0E94CA
:100C20000C062FEF84E39CE0215080409040E1F7D8
:100C300000C000000C946D1F0F931F93CF93DF93A0
:100C40008C0161E00E94F205EC01B8010E94BA0536
:100C5000882309F462C0B801CE010E94F5178823E9
:100C600009F45BC0B801CE010E94BC1C882309F4C2
:100C700054C0B801CE010E94EB18882309F44DC07E
:100C8000B801CE010E94181C882309F446C0F8015F
:100C900082818823D9F1CF3D8CE5D80779F140F4E2
:100CA000C115FCE5DF0791F0C130DC4591F02EC0A5
:100CB000CC35EDE5DE0741F1CD35FDE5DF0709F186
:100CC000CB35DD4519F50E94561120C00E940D0656
:100CD00024C080913102C82FC095C170C0FB80F93B
:100CE00080933102CC2329F088EC91E00E94140516
:100CF00014C086EB91E00E94140510C00E940412FB
:100D00000CC00E944D1102C00E945911C801DF9110
:100D1000CF911F910F910C94B605C0E08C2FDF91FD
:100D2000CF911F910F9108950E94A21E80E00E9412
:100D30002A180C94D1060E94AD160E94D4060C9479
:100D4000A81E8295982F937344E0949F90011124DC
:100D50008C7C86958695282B822F8575880F2A7A1C
:100D60002695822B089508950C94B30681E008958A
:100D7000CF93C82F0E94B606882329F0C0FD02C079
:100D80005E9A01C05E98CF910895569A5E9A089532
:100D9000CF93C82F0E94B4068C2F0E94B806CF9123
:100DA000089580E00C94C8060E94181D0C94C80693
:100DB000CF930E94181DC82F80918E01C81741F152
:100DC000C0938E018091310282FF1EC080FF04C05B
:100DD00080EE91E00E9414058091310280FF0CC0EA
:100DE0001F92CF938BED91E09F938F930E94AD055F
:100DF0000F900F900F900F908091310280FF04C0F0
:100E000089ED91E00E9414058C2FCF910C94C806B7
:100E1000CF910895CF93DF93CDB7DEB72B970FB661
:100E2000F894DEBF0FBECDBF4F83588769877A879E
:100E30008B8761110E9485109E012F5F3F4F86E0D6
:100E4000F90111928A95E9F785E0FE013796D901FB
:100E500001900D928A95E1F789819A814C815D819B
:100E6000452B31F09F3F31F491E08F3F19F403C0DF
:100E700091E001C090E090FF09C049815A816B81E7
:100E80007C818D819E810E94A60F05C0C9010E94B0
:100E9000FB058111F2CF2B960FB6F894DEBF0FBE83
:100EA000CDBFDF91CF910895FC01808191810E9497
:100EB000010D0895CF93882309F4A1C0C82F82386B
:100EC000C1F40E94181D81FD9AC069E3809102015E
:100ED000909103010E945D1E0E94A7102FEF81EEEA
:100EE00094E0215080409040E1F700C0000069E3A9
:100EF00019C0833801F50E94181D80FD80C063E58C
:100F000080910201909103010E945D1E0E94A71032
:100F10002FEF81EE94E0215080409040E1F700C037
:100F2000000063E580910201909103010E94681E18
:100F3000CF910C94A7108438C1F40E94181D82FD33
:100F40005EC067E480910201909103010E945D1EE2
:100F50000E94A7102FEF81EE94E021508040904036
:100F6000E1F700C0000067E4DDCF8CEF8C0F813A21
:100F7000F8F48C2F0E94CF1B811141C06C2F8091FF
:100F80000201909103010E94BB1D882349F06C2F40
:100F900080910201909103010E94681E0E94A71097
:100FA0006C2F80910201909103010E945D1EC0CFC1
:100FB00080E28C0F883048F4C77081E001C0880F50
:100FC000CA95EAF70E946810B3CFEBE5EC0FE33067
:100FD00040F4F0E0E15CFE4F808190E0CF910C9412
:100FE000791DC85AC73158F4EC2FF0E0EE0FFF1FFF
:100FF000EF5EFE4F80819181CF910C948F1DCF9138
:101000000895882309F45BC0682F823879F40E9420
:10101000181D81FF54C069E3809102019091030182
:101020000E945D1E0E94A71069E310C08338B1F4CE
:101030000E94181D80FF43C063E5809102019091DA
:1010400003010E945D1E0E94A71063E580910201CA
:10105000909103010E94681E0C94A710843879F4C3
:101060000E94181D82FF2BC067E4809102019091BD
:1010700003010E945D1E0E94A71067E4E7CF8CEF7A
:10108000860F813A18F380E2860F883048F4677043
:1010900081E001C0880F6A95EAF70E946E10DCCFEC
:1010A0008BE5860F833020F480E090E00C94791D6E
:1010B000685A673120F480E090E00C948F1D089509
:1010C0001F93CF93DF93182FEB010E945A072097AD
:1010D00041F08FE99FE00197F1F700C000002197F0
:1010E000F6CF812FDF91CF911F910C9401088933A6
:1010F00019F060E070E002C060E570E00C946008F8
:10110000882321F00E9468100C94A710089588236A
:1011100021F00E946E100C94A7100895CF92DF92D8
:10112000EF92FF920F931F93CF93DF937C01D62F03
:10113000C72FFC011281058102950F700E945E107D
:101140008823B9F01123A9F08C2F807F803421F0FF
:1011500080E28D0F883068F080916B0282FD09C0BB
:1011600082E00E9407110E945E1091E0D82ED926DD
:1011700001C0D12CCC2EC2948FE0C8228C2D90E0DF
:101180008C30910508F0C4C1FC01EA5AFF4F0C9461
:1011900063278C2F807FCF70882311F0C295C07F8A
:1011A000112399F0CC2309F49FC180E28D0F883080
:1011B00010F0D11104C08C2F0E94681003C08C2F36
:1011C0000E9478100E94A7108FC18D2F0E940108E5
:1011D000CC2309F49DC180E28D0F883038F1DD23E6
:1011E00029F18C2F0E947E1024C08C2F807FCF701D
:1011F000803211F0C295C07FDD2319F0D130A1F10A
:101200003DC080916B0282FF17C0112349F0CC23AF
:1012100029F08C2F0E9468100E94A71080E065C101
:1012200080E00E940108CC2309F472C18C2F0E9437
:101230006E100E94A7106CC1112371F0002341F0C1
:10124000013031F40E9488108C2B0E94901060C1F4
:101250000E9488108C2B1DC0002319F0013009F466
:1012600057C10E949D1025C0112321F0063008F0BF
:101270004FC10EC0053008F04BC11BC0112361F0F7
:10128000002331F0F701858180FF2EC18F708583A7
:101290008C2F0E9480083CC1002359F0D93309F0FB
:1012A00034C1FFEF07EE13E0F15000401040E1F7CA
:1012B0002AC18C2F0E9487082BC18C2F869586957A
:1012C000837019F0813061F023C1112321F08D2F3B
:1012D0009C2F937002C080E090E00E94791D20C195
:1012E000112321F08D2F9C2F937002C080E090E09D
:1012F0000E948F1D15C18C2F837009F047C01111FA
:101300000BC12D2F229526952770220F220F6D2FAE
:101310006F70862F90E0A0E0B0E0022E04C0880F2E
:10132000991FAA1FBB1F0A94D2F7D4FF10C04FE029
:1013300050E060E070E004C0440F551F661F771F47
:101340002A95D2F7409550956095709503C040E07E
:1013500050E0BA01C695C695C3708A019B01082B5F
:10136000192B2A2B3B2BC901B801C23049F058F484
:10137000C13019F00E94800BCFC00E946E0BCCC010
:101380000E94920BC9C00E946C0BC6C0112319F0B9
:101390008C2F817001C08695882309F4BDC02D2F44
:1013A000229526952770220F220F6D2F6F70862FA2
:1013B00090E0A0E0B0E0022E04C0880F991FAA1FA1
:1013C000BB1F0A94D2F7D4FF10C04FE050E060E09A
:1013D00070E004C0440F551F661F771F2A95D2F78F
:1013E000409550956095709503C040E050E0BA017B
:1013F000C695C695C3708A019B01082B192B2A2B11
:101400003B2BC901B801C23049F058F4C13019F082
:101410000E94450C81C00E94330C7EC00E94570C74
:101420007BC00E94A60B78C0CF70112339F08C2F9F
:101430000E94CC0B8D2F0E9480086EC08D2F0E94C1
:1014400087088C2F0E94ED0B67C0D23F21F128F452
:10145000D03F41F0D13FC1F043C0D33F19F1D43F59
:1014600079F03EC0112341F0053008F051C08C2FB7
:101470008F710E94120C4CC0063008F049C0F7CFA3
:1014800080916B0282FF18C0112339F08C2F8F716D
:101490000E94CC0B3DC01123C9F38C2F8F710E9489
:1014A000ED0B36C0112329F08C2F8F710E94B70BE2
:1014B0002FC00E94B20B2CC0112349F0CF718C2F8A
:1014C0000E94CC0B63E08C2F0E94EC1021C081E0C5
:1014D0000E9407110230E0F082E00E94071118C05C
:1014E000112331F0002391F28D2F0E945A0710C072
:1014F000002399F2D93349F41FEF27EE33E011505E
:1015000020403040E1F700C000008D2F0E9401080C
:1015100088EF8C0D843020F40E94181D0E94C806AC
:10152000DD20C9F00E945A1080FD15C0F70112821B
:101530000E9454100E94CC0BC7010E94CC0A0E944A
:101540005410DF91CF911F910F91FF90EF90DF909A
:10155000CF900C94ED0BDF91CF911F910F91FF90E5
:10156000EF90DF90CF9008950F931F93CF93DF9369
:10157000EC01688179818A810E940C0D8C010E94A6
:10158000690C0E945A0BB801CE010E948E08DF91AF
:10159000CF911F910F910895CF93DF93EC01988124
:1015A00089812B813C81232B31F08F3F31F481E005
:1015B0009F3F19F403C081E001C080E080FD1DC0A1
:1015C000CE010E941C06811110C00E945E1088236B
:1015D000A1F08A81882389F080916B0282FD0DC081
:1015E00082E0DF91CF910C940711CE010E94B40AE2
:1015F000CE01DF91CF910C94FD05DF91CF9108953D
:1016000080E090E00E94791D80E090E00E948F1DB4
:101610000E9485100C94A710809102019091030103
:101620000E94731E0C94000B0E9475100C940C0BFE
:1016300092959F70963079F010F4925001C09A50B4
:10164000923068F4803F69F018F4883E40F409C095
:10165000843F29F406C0883E20F0813F11F080E0ED
:10166000089581E00895FC01808191810E94010D1F
:101670000E94180B0895CF93DF9300D000D01F92E3
:10168000CDB7DEB70F900F900F900F900F90DF91B6
:10169000CF910895CF93DF9300D000D000D0CDB785
:1016A000DEB726960FB6F894DEBF0FBECDBFDF9132
:1016B000CF910895089508950C945B0B0C945C0BE6
:1016C0000E945E0B6093A3017093A4018093A50117
:1016D0009093A6010C94000B0C94600B0F931F9336
:1016E0000091A3011091A4012091A5013091A601C0
:1016F000602B712B822B932B1F910F910C94600BFD
:101700000F931F930091A3011091A4012091A501B3
:101710003091A60160237123822393231F910F919F
:101720000C94600B0F931F930091A3011091A401DF
:101730002091A5013091A601602771278227932768
:101740001F910F910C94600B0C945B0B0E94A40BE7
:1017500060939F017093A0018093A1019093A201D7
:101760000C94000B60E070E0CB010C94A60B0F937F
:101770001F9341E050E060E070E08A019B0104C0EB
:10178000000F111F221F331F8A95D2F7C901B8011C
:101790001F910F910C94A60B0F931F9341E050E003
:1017A00060E070E004C0440F551F661F771F8A95E4
:1017B000D2F780919F019091A001A091A101B091D9
:1017C000A2018A019B01082B192B2A2B3B2BC90153
:1017D000B8011F910F910C94A60B0F931F9341E03A
:1017E00050E060E070E004C0440F551F661F771F93
:1017F0008A95D2F7409550956095709580919F019C
:101800009091A001A091A101B091A2018A019B0138
:10181000082319232A233B23C901B8011F910F91E3
:101820000C94A60B0F931F9341E050E060E070E032
:1018300004C0440F551F661F771F8A95D2F7809109
:101840009F019091A001A091A101B091A2018A01F4
:101850009B01082719272A273B27C901B8011F9197
:101860000F910C94A60B0F931F9300919F01109161
:10187000A0012091A1013091A201602B712B822B3C
:10188000932B1F910F910C94A60B0F931F93009114
:101890009F011091A0012091A1013091A20160232C
:1018A0007123822393231F910F910C94A60B0F9306
:1018B0001F9300919F011091A0012091A1013091EF
:1018C000A20160277127822793271F910F910C9403
:1018D000A60B0895990F990F890FE82FE695E695C5
:1018E000E695877051E001C0550F8A95EAF785E0CB
:1018F000E89FF0011124E057FE4F20E030E070E057
:101900004081CB01022E02C0969587950A94E2F79A
:101910008170819584278523842781932F5F3F4F92
:101920002530310569F70895990F990F890F682FB0
:10193000669566956695982F977085E0689FB001CB
:10194000112440E050E080E0FB01E40FF51FE05778
:10195000FE4F208130E0092E02C0369527950A946B
:10196000E2F721703327042E01C0220F0A94EAF710
:10197000822B4F5F5F4F4530510531F70895BF927D
:10198000CF92DF92EF92FF920F931F93CF93DF934B
:101990008C01C0909F01D090A001E090A101F09037
:1019A000A2018091A3019091A401A091A501B09101
:1019B000A601C82AD92AEA2AFB2ACFE1D0E0D7011A
:1019C000C6010C2E04C0B695A795979587950A94E5
:1019D000D2F780FD04C0219790F7B12C07C0BC2E30
:1019E000B8018C2F0E94F6130197A9F38B2DDF917C
:1019F000CF911F910F91FF90EF90DF90CF90BF900C
:101A00000895CF93DF93EC010E94BF0CBE010E94AA
:101A1000F613DF91CF9108951F93CF93DF93EB01DE
:101A200090918F01992321F0CB010E94010D13C0E9
:101A3000882349F0CB010E94BF0C182F682FCE01DC
:101A40000E946A0C04C0CB010E94940C182FBE01A6
:101A5000812F0E94F613DF91CF911F9108951F935C
:101A6000CF93DF93C091A70116E08091A801C8171A
:101A700099F0D0E01C9FF0011D9FF00D1124E75557
:101A8000FE4F4081518162817381848195810E94E2
:101A90004A0B2196C770E9CFDF91CF911F9108952E
:101AA0004091D9015091DA016091DB017091DC0124
:101AB0008091DD019091DE010C944A0BEF92FF9230
:101AC0000F931F93CF93DF938091DE0182958F70E8
:101AD00009F065C08091DB01882309F460C0809122
:101AE000A701F090A8011091D9010091DA0160914D
:101AF000DC017091DD0191E01F3F09F090E0C091A1
:101B00000001D0910101292F96E0E92E8F1509F4EB
:101B100046C06115710521F00F3F21F030E003C090
:101B200031E001C0322F90E030FD36C0E89EF00178
:101B3000E99EF00D1124DF01A755BE4F11963C918F
:101B40001197301329C03C91311326C012963C9155
:101B50001297311121C013964D915C911497461B39
:101B6000570B4C175D07C0F48091DE018F708061C8
:101B70008093DE01E255FE4F80818F70806180830B
:101B800089ED91E00E94CC0ADF91CF911F910F91D6
:101B9000FF90EF900C942F0D01968770B7CFDF91D7
:101BA000CF911F910F91FF90EF9008959F92AF9268
:101BB000BF92CF92DF92EF92FF920F931F93CF933A
:101BC000DF93CDB7DEB761970FB6F894DEBF0FBED7
:101BD000CDBF8C0185E0F801DE011D9601900D92CC
:101BE0008A95E1F7D8011296EC909091D901E09195
:101BF000DA012091DC013091DD012115310531F050
:101C0000EF3F31F481E09F3F19F403C081E001C050
:101C100080E0B82FB1709B2E80FD47C1D8014C9158
:101C200011965C9111971396AD90BC90149789ED25
:101C3000C82E81E0D82EF090DB01B501621B730B3A
:101C40002091000130910101FF2009F4D9C0809159
:101C5000DE016217730708F095C0282F207F09F076
:101C600052C05E1313C0491311C0FE2CE1100EC008
:101C70008F7080618093DE010E94500DC6010E942A
:101C8000CC0A8091DE01F80185834DC1AB2831F08B
:101C90005F3F31F481E04F3F19F403C081E001C0A0
:101CA00080E080FD03C081E08E2502C080E090E0EE
:101CB000F82FF170FF2E80FF1CC08091A7012091AA
:101CC000A80136E0821709F40BC190E0389FF001BB
:101CD000399FF00D1124E755FE4F6181561306C060
:101CE0006081461303C06281E61203C001968770CB
:101CF000E9CFFE2CEE2009F416C18091DE0181604F
:101D00008093DE0154C05E1306C0491304C0E11085
:101D100002C0F80199C0C8010E94330B882361F109
:101D2000EE2051F12091DE01822F82958F7090E09C
:101D3000029774F08091D9019091DA0198878F838E
:101D40001986BB86AA862C87CE0107960E94CC0AEC
:101D500086E0F801A9EDB1E001900D928A95E1F7D6
:101D60000E945E0D0E94500D0AC05E1711F1C8015D
:101D70000E94330B81112CC0C8010E94CC0AFF24A1
:101D8000F394D1C0282F207F81F77A2DB98AA88AB1
:101D90006E2D89890E943B0B89ED91E00E94CC0A4F
:101DA00086E0D6011D928A95E9F70E94500DF12C2C
:101DB000BAC04913DCCFE110DACFF8018583C8013E
:101DC0000E94CC0A86E0D6011D928A95E9F7ABC045
:101DD000EE2091F22091DE01822F82958F7090E0AB
:101DE00002970CF4B5CF8091D9019091DA019A83D2
:101DF00089831B82BD82AC822E83CE010196A6CF41
:101E00006217730708F044C0FE2CEE2009F4B4CF2B
:101E10005E1330C049132EC02091DE0120FD21C089
:101E2000822F82958F70482F50E041155105C9F0DF
:101E3000F80125834F30510541F08F5F982F92951F
:101E4000907F822F8F70892B8583C8010E94CC0AD6
:101E500086E0F801A9EDB1E001900D928A95E1F7D5
:101E60003CC086E0F801A9EDB1E001900D928A95A1
:101E7000E1F759C0C8010E94330B811169CF8091ED
:101E8000DE0181608093DE01C8010E94CC0A4BC054
:101E90007A2DB98AA88A6E2D89890E943B0B86E02B
:101EA000D6011D928A95E9F718C0EE2009F464CF97
:101EB000C8010E94330BF82E882309F45DCF86E019
:101EC000F801A9EDB1E001900D928A95E1F789ED55
:101ED00091E00E9454070E945E0D0E94500D23C0A5
:101EE0004D875E878D859E850E94010D292F229545
:101EF0002F70223028F49F7039F0811105C00BC07B
:101F0000243028F49F7049F4805E883020F0C801A6
:101F10000E94CC0A9F2CF92C06C0D80115969C91E2
:101F2000907F91F7F8CF8F2D61960FB6F894DEBFB2
:101F30000FBECDBFDF91CF911F910F91FF90EF901A
:101F4000DF90CF90BF90AF909F9008951F93CF9355
:101F5000DF93CDB7DEB72C970FB6F894DEBF0FBE78
:101F6000CDBF4F83588769877A878B879C87CE013F
:101F700007960E94D60D8823D1F09F8188852A85F7
:101F80003B85232B31F08F3F31F481E09F3F19F4E3
:101F900003C081E001C080E080FD47C04F815885CB
:101FA00069857A858B859C850E944A0B3EC086E0B8
:101FB000FE013796DE01119601900D928A95E1F7A8
:101FC000FF81E8856A857B856115710531F0EF3FFA
:101FD00031F481E0FF3F19F403C081E001C080E0EB
:101FE00080FD23C02091A80130E0C90101968770CF
:101FF00099274091A70150E084179507F1F1F983E3
:10200000EA837D836C8396E0929FD001939FB00D0D
:102010001124A755BE4FFE01319601900D929A955D
:10202000E1F78093A8010E942F0D16E08091A7018F
:102030009091A801891771F1189FC001112487554B
:102040009E4F0E94D60D882329F1E091A7011E9F83
:10205000F0011124E755FE4F408151816281738167
:10206000848195810E944A0B8091A70190E001969E
:10207000877099278093A701D9CF0E94140B1092E3
:10208000A8011092A701E9EDF1E086E0DF011D92C1
:102090008A95E9F72C960FB6F894DEBF0FBECDBF38
:1020A000DF91CF911F9108958091FF0185958595CE
:1020B000859508958091FF01877008959091FF01A3
:1020C000977081E009F480E00895809122020895DC
:1020D00090912202892B80932202089580959091FD
:1020E00022028923809322020895109222020895E9
:1020F00090912102892B80932102089580959091DF
:1021000021028923809321020895109221020895CB
:1021100080910002089508950C948B100C948C10FB
:1021200090916B0292FD08C090910002981721F0E7
:10213000809300020C948E100895809100028823F1
:1021400029F01092000280E00C948E100895CF9335
:10215000DF93E0910201F0910301809122028083DC
:10216000E0910201F0910301908180912102892B7D
:10217000808380910002882381F0E0910201F09138
:1021800003019081892B808380910201909103014A
:102190000E94A51D81110E949D10C0910201D09145
:1021A000030140E250E06FED71E0CE010E94832711
:1021B000892B69F080E2FE01AFEDB1E001900D9254
:1021C0008A95E1F7CE01DF91CF910C94241DDF9128
:1021D000CF9108950C948B1090916B0292FD10C0DA
:1021E00098E0899F90011124262B2093FF010E94E3
:1021F000CC0B8091FF018595859585950C94EA100F
:102200000C94CC0B1092FF0180E00C94EA1020910A
:10221000FF01809582238093FF01982F977099F496
:1022200030E0482F082E000C550B2417350759F0C5
:1022300090916B0292FD07C08595859585950E94CA
:10224000ED0B0C9402110895CF9390916B0292FBC9
:10225000222720F92817F9F0C82F892FC0FB82F90F
:1022600080936B0280916A0290916B020E948011B0
:1022700082E00E9407118091310280FF0CC01F9202
:10228000CF938BEE91E09F938F930E94AD050F90BB
:102290000F900F900F90CF91089580916B0282FB69
:1022A000882780F991E089270C94241181E00C940F
:1022B000241180E00C94241180E090E00E94982783
:1022C00021E0893E9E4F09F020E0822F089582E0B0
:1022D00090E00C94902783E090E00C949027CF93AB
:1022E00084E090E00E949027C82F82E290E00E9454
:1022F00090272C2F30E0A901582BCA01CF910895C7
:10230000CF93C92F682F84E090E00E949E276C2F06
:1023100082E290E0CF910C949E27AB01BC018FE04C
:1023200090E00C94B027AB01BC0183E190E00C94E9
:10233000B02760E070E0CB010C94931160E070E096
:10234000CB010E948D110C94991169EE7EEF80E013
:1023500090E00E94BC2760E082E090E00E949E270F
:1023600060E083E090E00E949E271092A30110920B
:10237000A4011092A5011092A60160E084E090E013
:102380000E949E2760E082E290E00E949E2760E02B
:1023900085E090E00E949E2760E086E090E00E9449
:1023A0009E276FEF87E090E00E949E2740E050E07C
:1023B000BA0188E090E00E94B02760E08DE090E0F4
:1023C0000E949E2740E050E0BA0188E190E00E9420
:1023D000B02760E087E190E00E949E2740E050E057
:1023E000BA018CE190E00E94B02760E070E080E2EA
:1023F00090E00E94BC2740E050E0BA0188E190E004
:102400000E94B0270C949E110C94A511682F8EE0A9
:1024100090E00C949E270E942C1F60932D027093D5
:102420002E0280932F0290933002609329027093C2
:102430002A0280932B0290932C02089585B780681E
:1024400085BF85B7806885BF089581E008950C94A5
:10245000251208950C9429120C9429120C942C1214
:102460000C9429120C9430120C9429120E941E1202
:102470008BE591E20E940E1D0E9434120C943212E0
:102480000E942A120C9429120E94D3140E94C5069D
:102490000C94DB180E94171F0E94EF150E94441233
:1024A0000E94AD160C942E128F929F92AF92BF9203
:1024B000CF92DF92EF92FF920F931F93CF93DF9310
:1024C000CDB7DEB72A970FB6F894DEBF0FBECDBFEB
:1024D0000E940416982E81110E940B1283E2A82EEE
:1024E00082E0B82E00E010E0802E802F0E94F714CA
:1024F000D82EF501C1905F01C826B1F40F5F1F4FC0
:102500000630110589F78FEF89838A831B820E9429
:10251000201F8160782F9D838C8349815A816B8134
:102520008D810E940A072FC08091310281FD0E9497
:10253000FD14E12CFF24F3948C2D8F21F1F00E94E7
:102540002712882399F0EE828F82DF2081E009F440
:1025500080E088870E94201F8160782F9A87898772
:102560004E815F8168858A850E940A07F801ED5DCA
:10257000FD4F8081F826F08206C0E394FF0CF4E062
:10258000EF12DACFBBCF81E0911001C080E02A9634
:102590000FB6F894DEBF0FBECDBFDF91CF911F9174
:1025A0000F91FF90EF90DF90CF90BF90AF909F90F2
:1025B0008F9008950E9454120E94DA180C94D80645
:1025C000CF93DF930E94FB13EC01811522E5920764
:1025D000E8F5811531E5930708F0B6C0883E91050E
:1025E00028F5803E910508F0E9C0883A910570F41D
:1025F000853A910508F07AC08130910509F473C0DD
:1026000008F4D9C0049708F0D9C0D5C08F3B910514
:1026100008F0D1C0C85AD0E0CC0FDD1FCE5BDE4F32
:102620000990D881C02DCE019464C9C0811540E5C0
:10263000940708F069C0811550E4950708F060C060
:102640009A9581159F4108F4B9C0B5C0811536E54A
:10265000930728F5811545E5940708F092C0811588
:1026600054E5950708F087C0AC0143705527282F23
:1026700026952695C115D34508F06CC081E090E001
:1026800002C0880F991F4A95E2F740E2249F90010B
:102690001124EC01C22BD32BCE019C6890C0811574
:1026A0002AE5920780F4811539E5930708F072C096
:1026B000811548E5940708F47EC0D82FCC27CE01B9
:1026C000806F906A7CC090568115904208F073C06C
:1026D0008D2F8F710E948F14DD27D0628F71AE0114
:1026E000582BCA016CC081E090E069C0C55AD0E0A7
:1026F000C059DE4F8881C82FD0E0CE0190645FC002
:10270000DF70CE01906A5BC074E0969587957A95EC
:10271000E1F7282F23703C2F337081E090E002C056
:10272000880F991F3A95E2F79C68AC01522B9A01E9
:102730009C2F9F709695969550E2959FE0011124ED
:10274000C9018C2B9D2B3BC0D82FCC27CE01816F8C
:10275000906A35C081E090E002C0880F991F4A95C9
:10276000E2F750E2259F90011124EC01C22BD32BFC
:10277000CE019A6824C0D82FCC27CE01846F906AEE
:102780001EC00E948F148F7190E0D82FCC27CE01ED
:10279000906215C08F700E948F1494E0D695C795F3
:1027A0009A95E1F7CF70D0E0DC2FCC27D0699E015D
:1027B000282BC90104C080E090E001C0CE01DF9168
:1027C000CF910895E72FF0E096E0899FE00DF11D8D
:1027D0001124EE0FFF1FEE0FFF1FE60FF11DEE0F8E
:1027E000FF1FEA5AFE4F8591949108950E94E213CB
:1027F0000E94E01208958238910569F1B0F48133A6
:10280000910509F46DC048F48932910509F463C05B
:102810008A32910509F469C008958533910509F458
:1028200055C089339105B9F00895833E910569F14A
:1028300038F4803E9105B1F0823E910509F108958A
:10284000863E9105A9F1873E9105B9F1843E910537
:1028500009F064C023C020916A0220FD4FC021FD11
:102860004DC0089580916A0280FD44C080916B0242
:1028700080FF44C080916A0284FD42C083EE4DC057
:1028800080916A0282FF38C0F5CF80916A0282FD92
:1028900033C080916B0280FD31C0ECCF80916B0220
:1028A00081FF32C080916A0284FD2AC087EE35C064
:1028B00080916A0283FF26C0F5CF80916A0283FD72
:1028C00021C080916B0281FD1FC0ECCF80916A0214
:1028D00085FD1CC01DC080916A0285FD19C016C00F
:1028E00080916A0286FD16C017C080916A0286FD3B
:1028F00013C010C089E311C082EE0FC080EE0DC07E
:1029000080E00BC086EE09C084EE07C089E205C0F6
:1029100085E303C08AE201C081E390E008959091CD
:102920006A0292FF0DC0282F2871283019F4877F82
:10293000846006C0282F2471243011F48B7F8860B6
:1029400093FF0DC0282F2871283119F4877E8461E8
:1029500006C0282F2471243111F48B7E88612091C8
:102960006B0220FF0DC0382F3871383019F4877F83
:10297000816006C0382F3171313011F48E7F88604C
:1029800021FF0DC0282F2871283119F4877E81611D
:1029900006C0282F2171213111F48E7E886194FDAB
:1029A000877E089508950E945C11811102C00E94E3
:1029B00004120E946711809331020E946F1190935C
:1029C0006B0280936A020E94D2140E946B11682FDE
:1029D00070E080E090E00E946C0B60919F0170912C
:1029E000A0018091A1019091A2010C94A40BE82F69
:1029F000F0E0EE58FD4F80810895CF92DF92EF9284
:102A0000FF920F931F93CF93DF938FE092E00E948A
:102A1000140582E7E82E82E0F82EC0E0D0E09AE0CC
:102A2000C92E92E0D92E02E012E0DF93CF93DF921D
:102A3000CF920E94AD0587E092E00E941405F70155
:102A400081917F010E94A1061F928F931F930F9384
:102A50000E94AD0580E092E00E94140521968DB79A
:102A60009EB708960FB6F8949EBF0FBE8DBFC630B6
:102A7000D105D9F6DF91CF911F910F91FF90EF9083
:102A8000DF90CF90089580EA8A95F1F7089500C00D
:102A900008950C94431508950C944B150C944C1503
:102AA0000C944B150C945015F894E82FE295EF70A8
:102AB000F0E031A1282F2F7081E090E001C0880F55
:102AC0002A95EAF7982F9095932391A392A1892BA9
:102AD00082A3789408950F931F93CF93DF93C7E752
:102AE000D1E089918F3F11F00E94541581E0CD37DC
:102AF000D807B9F7C3E7D1E007E711E089918F3F25
:102B000011F00E9454150C171D07C1F7DF91CF91EA
:102B10001F910F910895CF92DF92EF92FF920F9342
:102B20001F93CF93DF938C01C62FD0E0CE0189583D
:102B30009E4F7C01FC0190819F3F09F447C0D62E37
:102B4000F894E92FE295EF70F0E081A19F7021E009
:102B500030E001C0220F9A95EAF7822B81A382A16F
:102B60002095282322A378940E944715E3E7F1E0FB
:102B700047E751E031E0C12C21912F3F89F0A22F8E
:102B8000A295AF70B0E090968C9190E02F7002C04B
:102B9000959587952A95E2F780FD02C0832F01C0A5
:102BA00080E0C82A330F4E175F0731F7F7018081A5
:102BB0008F3F11F00E94541561E0C11001C060E028
:102BC0008D2D0E944915C00FD11FC882DF91CF9172
:102BD0001F910F91FF90EF90DF90CF9008950E948A
:102BE0006B1586E0E2E7F2E0DF01982F1D929A95DF
:102BF000E9F7ECE6F2E0DF011D928A95E9F786E05D
:102C00000E944C160C940806FF920F931F93CF93CB
:102C1000DF9300D000D000D0CDB7DEB78E010F5FBC
:102C20001F4F86E0F80111928A95E9F7F12C6F2D7C
:102C3000C8010E948B15F394F6E0FF12F8CF46E02E
:102C400050E0B8018CE692E00E948327FF24F394C1
:102C5000009709F4F12C892B41F086E0F801ACE6ED
:102C6000B2E001900D928A95E1F72F2D46E062E7E0
:102C700072E08CE692E00E944D160E940A068F2DAB
:102C800026960FB6F894DEBF0FBECDBFDF91CF9171
:102C90001F910F91FF9008950895FF920F931F9336
:102CA000CF93DF938C01F62ED72FC42F222349F028
:102CB00081E0809334020E94201F9093330280931E
:102CC0003202809134028823C1F0809132029091C7
:102CD00033020E94381F059780F0EF2DFD2FD80199
:102CE0004C2F50E0CD01801B910B841795071CF4ED
:102CF0008D918193F7CF10923402DF91CF911F9184
:102D00000F91FF9008950E94D7210E944A120C94BF
:102D1000E3210E94E7210E94DA120C9405220E940E
:102D2000BE1E0E94BE210E9436120E9483160E947F
:102D300089160E944012FBCF86E090E00C94902709
:102D4000682F86E090E00C949E2780917802847032
:102D50008162809378020C94A0160E945C1181110C
:102D600004C00E9404120E94A5160E949C16809323
:102D70007802282F26952695269530E025303105B6
:102D800024F087708062809378028091780280FFBF
:102D900004C086958695869501C080E00C942A181B
:102DA00020917802822F869586958695482F50E04F
:102DB0004430510554F48F5F982F990F990F990F54
:102DC000822F8770892B80937802809178028160AE
:102DD000809378020E94A0168091310280FF11C07A
:102DE000809178028695869586951F928F9385E8C7
:102DF00092E09F938F930E94AD050F900F900F90DC
:102E00000F90809178028695869586950C942A1865
:102E100080917802982F969596959695A1F0915E5F
:102E2000990F990F990F8770892B80937802887F6B
:102E300091E009F490E08091780290FB80F9809312
:102E400078020E94A0168091310280FF11C080910B
:102E500078028695869586951F928F938DE692E0EF
:102E60009F938F930E94AD050F900F900F900F903E
:102E7000809178028695869586950C942A18809183
:102E8000780280FD1FC0816080937802813019F440
:102E900089E080937802809178020E94A016809148
:102EA000310280FF08C085E492E09F938F930E94D7
:102EB000AD050F900F908091780286958695869546
:102EC0000C942A1808958091780280FF14C08E7F98
:102ED000809378020E94A0168091310280FF08C082
:102EE00082E392E09F938F930E94AD050F900F9025
:102EF00080E00C942A180895CF93C0917802C17095
:102F00008091310280FF0CC01F92CF9387E592E041
:102F10009F938F930E94AD050F900F900F900F908D
:102F2000CC2319F0CF910C946317CF910C943F17D9
:102F300090917802892F8695869586958F5F8F71FF
:102F40009770853038F4880F880F880F892B80930D
:102F5000780202C09093780280917802887F91E095
:102F600009F490E08091780290FB80F980937802D8
:102F70000E94A0168091310280FF11C080917802DA
:102F80008695869586951F928F938EE192E09F930A
:102F90008F930E94AD050F900F900F900F9080912E
:102FA00078028695869586950C942A18853008F0C7
:102FB00084E0909178029770282F220F220F220F21
:102FC000922B90937802987F21E009F420E0909171
:102FD000780220FB90F9909378020C942A180E94B2
:102FE000D617809178020C94A0169C01FB01828177
:102FF000882349F12E3BFCE53F07C9F040F42C3B08
:10300000ECE53E0769F02D3B3C4561F00895203C1E
:103010009CE5390791F070F0213C3C4589F008951A
:1030200084E001C080E00E94EF1780E008950E94D4
:103030000817FBCF0E94D016F8CF0E947C17F5CF5F
:103040000E949817F2CF81E00895269A2E9808954D
:103050002E9808958F929F92AF92BF92CF92DF9257
:10306000EF92FF920F931F93CF93DF93C82F85307A
:1030700050F4811109C0809180008F7D8093800081
:103080000E94281806C0C4E080918000806280936E
:103090008000A0918600B09187002C2F30E00E9424
:1030A00069278B019C0142E0369527951795079576
:1030B0004A95D1F780918600909187006CE070E08E
:1030C0000E942D276017710730F0C80169E070E099
:1030D0000E942D275EC08091860090918700E0902D
:1030E0008600F0908700E0918600F0918700C6E0AE
:1030F000D0E0BE010E942D27060F171F211D311D94
:103100004801590185E0880C991CAA1CBB1C8A95B2
:10311000D1F7C701BE010E942D276F01E12CF12CD0
:10312000A7019601260F371F411D511DC501B4018E
:103130000E94412769017A01E0918600F0918700A1
:10314000CA01B9010E9411279B01AC01DF010E9455
:1031500078279B01AC01C701B6010E941127DC0151
:10316000CB012FE0B695A795979587952A95D1F72E
:10317000009186001091870020E030E008171907C1
:103180002A073B0728F46091860070918700CB01E5
:10319000BC0170938B0060938A00DF91CF911F91E7
:1031A0000F91FF90EF90DF90CF90BF90AF909F90E6
:1031B0008F90089508950E94251882E280938000E0
:1031C00089E1809381008FEF9FEF90938700809338
:1031D00086000C94AD16CF93DF93EC01FB01828146
:1031E000882309F43CC1C430FDE5DF0760F4CB3F20
:1031F0009CE5D90788F49E0122503C4524313105D5
:1032000008F02EC109C0C236EDE5DE0729F0C63A46
:10321000FDE5DF0709F024C10E946F1190936B0256
:1032200080936A02C1318CE5D80709F4C6C008F062
:1032300042C0C930ECE5DE0709F49BC000F5C5309B
:103240008CE5D80709F485C078F4C330ECE5DE07D7
:1032500009F478C008F07AC0C230DC4509F0F5C046
:1032600080916A028160EFC0C7309CE5D90709F4FC
:1032700078C008F07AC080916A028061E4C0CD30E5
:10328000FCE5DF0709F487C058F4CB309CE5D9078B
:1032900009F479C008F07BC080916A0288606FC031
:1032A000CF30FCE5DF0709F480C008F082C08091D0
:1032B0006A02877FC8C0CE3F9CE5D90709F471C078
:1032C00000F5C531FCE5DF0709F485C068F4C331BA
:1032D0009CE5D90709F475C008F095C00E94140B4D
:1032E00080916A028F77AFC0CC3FFCE5DF07A9F180
:1032F00008F054C0CB3FDC4509F0A7C080916B02B9
:1033000040C0C230EDE5DE0709F489C058F4C115AC
:103310008DE5D80709F45AC008F069C080916B02A6
:1033200082602FC0C236EDE5DE0709F47CC0C63AE4
:10333000FDE5DF0709F481C0C330DD4509F085C034
:1033400080E06EC080916A0282607DC080916A02D6
:1033500016C080916A02886076C080916B0282609C
:103360004FC080916A0280626EC080916A02806460
:103370006AC00E94140B80916A02806864C08460F5
:1033800062C081603DC080916A028E7F5CC0809186
:103390006A028D7F58C080916A0216C080916B02CC
:1033A00018C080916B028D7F2BC080916A028F7E46
:1033B0004AC080916A028F7D46C080916A028F7BED
:1033C00042C080916A02877F8B7F3DC080916B02F3
:1033D0008D7F8E7F15C080916A0282FB222720F9A3
:1033E00091E0922790FB82F990FB83F92CC08091A9
:1033F0006B02982F909591708E7F892B90FB81F9AD
:1034000080936B0222C00E94140B80916A0287FB9A
:10341000222720F991E0922790FB87F914C081E0E0
:103420000E94061212C080916A0284FB222720F9B2
:1034300091E0922790FB84F906C080916A02982F50
:10344000909590FB80F980936A0280916A02909136
:103450006B020E9480110E94140B80E001C081E089
:10346000DF91CF910895CF93C82F1F928F9383EA56
:1034700092E09F938F930E94AD0581E090E0A0E0E1
:10348000B0E0BC01CD0104C0660F771F881F991FF3
:10349000CA95D2F70E946C0B0F900F900F900F906F
:1034A000CF910C94140BDF92EF92FF920F931F9326
:1034B000CF93DF93482F50E0FA013597EF33F105B2
:1034C00008F05BC1EE59FF4F0C9463270E946B110B
:1034D0001F928F9388E097E09F938F930E94AD0592
:1034E0000E94671183FB992790F91F929F9382FB9B
:1034F000992790F91F929F9381FB992790F91F922A
:103500009F93982F91701F929F931F928F938FEB91
:1035100096E09F938F930E94AD050E946F1187FBE9
:10352000222720F91F922F9386FB222720F91F9232
:103530002F9385FB222720F91F922F9384FB2227AC
:1035400020F91F922F9383FB222720F91F922F939C
:1035500082FB222720F91F922F9391FB222720F92B
:103560001F922F93292F21701F922F9381FB2227C7
:1035700020F91F922F93282F21701F922F939F9332
:103580008F938AED95E09F938F930E94AD058DB741
:103590009EB788960FB6F8949EBF0FBE8DBF0E944F
:1035A0009C16982F9695969596951F929F93982F77
:1035B00091701F929F931F928F9387EA95E09F933C
:1035C0008F930E94AD058DB79EB708960FB6F894FD
:1035D0009EBF0FBE8DBF06C088EC97E00E94140509
:1035E0000E940412C1E0CEC085EF93E074C08091C8
:1035F0003102817F8E7F809331028AED93E00E94B9
:10360000140584EC97E00E94140581E08093350254
:10361000E9CF88EA97E00E9414050E940D06E2CFE8
:1036200080913102C82FC095C170C0FB80F9809392
:103630003102CC2319F08CE997E091C08FE897E034
:103640000E94140580913102897F877F8093310227
:10365000C9CF9091310291FBCC27C0F981E0C827F6
:10366000892FC0FB81F980933102CC2319F082E8C5
:1036700097E027C084E797E02EC09091310292FB3B
:10368000CC27C0F981E0C827892FC0FB82F980933D
:103690003102CC2319F085E697E013C085E597E069
:1036A0001AC09091310293FBCC27C0F981E0C82762
:1036B000892FC0FB83F980933102CC2351F089E438
:1036C00097E00E941405809131028160809331025D
:1036D00059C08CE397E00E94140584CF8CE293E0FC
:1036E000FACF0E942C1F062FF72EE82ED92EC0915C
:1036F0006A02C7FBCC27C0F910916902D091100172
:103700000E94181DDF92EF92FF920F931F92CF93AA
:103710001F921F931F92DF931F928F9388EA92E06C
:103720009F938F930E94AD058DB79EB70E960FB6EF
:10373000F8949EBF0FBE8DBF55CF0E94140B909181
:103740006A0297FBCC27C0F981E0C827892FC0FB0C
:1037500087F980936A02CC2329F082E397E00E94E4
:10376000140510C087E297E0B6CF895303C08D518E
:1037700001C080E00E94331A35CF85E297E00E94B5
:103780001405C0E08C2FDF91CF911F910F91FF9016
:10379000EF90DF90089580E008950C94CB1BCF93B9
:1037A000C82F80913502882319F0813031F038C05C
:1037B0000E9465108232B1F504C00E946510823209
:1037C00061F48C2F0E94CD1B811104C08C2F0E94AC
:1037D000531A24C081E090E021C08C2F0E94CB1BA3
:1037E00081111BC0C43189F018F4CB3029F010C00E
:1037F000C93259F0C83361F48AED93E00E94140590
:103800008FE992E00E94140508C0109235020CC0A6
:103810008DE992E00E94140507C081E0817006C026
:103820001092350280E002C080E0F8CFCF91089579
:10383000CF93DF9386319C4541F5EB010E946510E3
:10384000982F8A812091020130910301882379F019
:103850009A7A81E009F480E080933602911102C0E7
:1038600069E201C065E3C9010E945D1E0AC0809142
:103870003602811102C069E201C065E3C9010E94FC
:10388000681E0E94A71080E001C081E0DF91CF9107
:1038900008950F931F93CF93DF93C42FD22FFC0172
:1038A00082818823C9F0409339020E94201F90939F
:1038B00038028093370280E28C0F883008F057C0BE
:1038C000C77081E001C0880FCA95EAF7DF91CF91F8
:1038D0001F910F910C94800880913902481330C0D9
:1038E00080913702909138020E94381F883C9105E0
:1038F00038F510E21D0FCD17B9F080E28C0F88303B
:1039000040F4C77081E001C0880FCA95EAF70E94B1
:103910008708183028F581E09D2F977001C0880F27
:103920009A95EAF70E948008802F0E947708183045
:10393000F0F4D77081E001C0880FDA95EAF70AC089
:1039400080E28C0F883098F4C77081E001C0880F46
:10395000CA95EAF7DF91CF911F910F910C948708D8
:10396000802FDF91CF911F910F910C947708DF91F9
:10397000CF911F910F9108950F939C01CB01243F8C
:103980004CE5340731F188F4293DFCE53F07D9F0D7
:103990002A3D4CE5340779F1283D3C45A9F506E27E
:1039A00021EE41EE68ED7CE52BC0263FFCE53F07AC
:1039B000E1F0A8F0273F3C4539F507E225EE46EE59
:1039C00067EF7CE51DC007E225EE45EE69ED7CE57D
:1039D00017C006E221EE40EE64EF7CE511C007E27D
:1039E00025EE44EE65EF7CE50BC006E221EE42EEEB
:1039F00066EF7CE505C008E221E045EE6AED7CE576
:103A00000E94491C80E008C0FC018281882319F0D3
:103A10001092390201C081E00F91089590938D01B9
:103A200080938C01089590933F0280933E02089505
:103A3000E0913E02F0913F02309721F00190F08139
:103A4000E02D099480E00895EF92FF921F93CF93A9
:103A5000DF93FC01A0913E02B0913F02109709F460
:103A600042C080911001882341F080916A0287FF53
:103A700004C08081818386E08083EF011296ED91FE
:103A8000FC911397CE0109958091310282FF2BC0E2
:103A900080FF04C081EE97E00E94140518E08BEDD2
:103AA000E82E87E0F82E8091310280FF0BC08881DC
:103AB0001F928F93FF92EF920E94AD050F900F908F
:103AC0000F900F90115021961111EDCF809131027E
:103AD00080FF09C089ED97E0DF91CF911F91FF90A2
:103AE000EF900C941405DF91CF911F91FF90EF9010
:103AF000089520913C0230913D022817390771F05A
:103B000090933D0280933C02E0913E02F0913F028F
:103B1000309721F00680F781E02D099408952091D7
:103B20003A0230913B022817390771F090933B021B
:103B300080933A02E0913E02F0913F02309721F0EB
:103B40000084F185E02D09940895FC01329680915E
:103B50001001882331F080916A0287FF02C09EE144
:103B600001C096E080E0915028F021912223D9F302
:103B70008F5FF9CF0895662351F120911001222320
:103B8000E9F020916A0227FF19C0462F4695469515
:103B900046954E31E0F4677021E030E002C0220F1C
:103BA000331F6A95E2F7FC01E40FF11D828190E07A
:103BB0002823392381E0232B69F409C0FC013296C4
:103BC00008962191621729F0E817F907D1F780E0EC
:103BD000089581E008959C01FC0132969FEF80E0FA
:103BE0004191461789F09F3F19F4411101C0982F68
:103BF0008F5F8630A9F79F3F39F0F901E90FF11D7A
:103C000097FDFA956283089508959C012A5F3F4FBE
:103C1000FC014281461301C012820196821793076C
:103C2000B9F70895262F2695269526952E3170F4FE
:103C3000FC01E20FF11D677021E030E001C0220FAE
:103C40006A95EAF78281282B2283089580913102B8
:103C500080FF0CC01F926F9381E198E09F938F9338
:103C60000E94AD050F900F900F900F900895262F92
:103C70002695269526952E3178F4FC01E20FF11D4C
:103C8000677021E030E001C0220F6A95EAF72095C5
:103C900082812823228308958091310280FF0CC005
:103CA0001F926F9383EF97E09F938F930E94AD05D0
:103CB0000F900F900F900F900895209110012223E4
:103CC00029F020916A0227FD0C94121E0C94EB1D22
:103CD00020911001222329F020916A0227FD0C94E3
:103CE000371E0C94051E20911001FC0132962223F0
:103CF00031F080916A0287FF02C08EE101C086E048
:103D0000DF011D928A95E9F7089508950C94851EA8
:103D100083E0809340020C94861E811102C081E0F2
:103D200001C082E0809340020C94861E0C948D1E8C
:103D300081E0809340020C94861E0C94981E089596
:103D40000C949F1E0C94A01E0C949F1E0C949F1EFE
:103D50000C949F1ECF930E94A61E0E9404160E94E0
:103D6000A41EC0E08C2F0E94F714811104C0CF5F05
:103D7000C630C1F701C081E0CF91089508951F9228
:103D80000F920FB60F9211248F939F93AF93BF930F
:103D900080914102811113C08091790290917A0241
:103DA000A0917B02B0917C024196A11DB11D809330
:103DB000790290937A02A0937B02B0937C02BF9128
:103DC000AF919F918F910F900FBE0F901F901895FC
:103DD00080918102843031F10E9494061092410258
:103DE00020E488E190E00FB6F894A89580936000F5
:103DF0000FBE2093600083B7817F846083BF83B749
:103E0000816083BF7894889583B78E7F83BF0FB618
:103E1000F894A8958091600088618093600010926A
:103E200060000FBE08950E94140B0C949B0682E064
:103E300084BD93E095BD9AEF97BD80936E00089581
:103E40002FB7F8948091790290917A02A0917B0229
:103E5000B0917C022FBF08952FB7F894609179023A
:103E600070917A0280917B0290917C022FBF08951D
:103E70009C014FB7F8948091790290917A02A091B9
:103E80007B02B0917C024FBF821B930B0895789404
:103E90001F920F920FB60F9211248F939F93AF939F
:103EA000BF938091790290917A02A0917B02B091A8
:103EB0007C020196A11DB11D8093790290937A0234
:103EC000A0937B02B0937C02BF91AF919F918F91A1
:103ED0000F900FBE0F901F90189581E08093E00027
:103EE00080E28093D8001092C9008FE19EE4019790
:103EF000F1F700C0000087E090EBDC0180938A02BC
:103F000090938B02A0938C02B0938D029CE088E189
:103F10000FB6F894A895809360000FBE9093600050
:103F2000FFCF8091680208950895CF93DF93209189
:103F30001001222339F020916A0227FF03C060E2BA
:103F400022E002C068E021E02093E9002FEF3091E9
:103F5000E800215035FD06C035ED3A95F1F7000037
:103F60002111F5CF2091E80025FF1DC0EC018091C3
:103F70001001811105C040E050E068E070E003C02E
:103F800070E040E050E0CE010E9474228091E80091
:103F90008E778093E80080E2FE01A8E4B2E0019011
:103FA0000D928A95E1F7DF91CF91089580934402B5
:103FB000709346026093450280918102843001F53E
:103FC00082E08093E9008FEF9091E800815095FDA9
:103FD00006C095ED9A95F1F700008111F5CF80911B
:103FE000E80085FF0DC040E050E063E070E084E44D
:103FF00092E00E9474228091E8008E778093E8001E
:104000000895BC0184E00C94D61FBC0183E00C949D
:10401000D61F089583E498E00E94140580918002E1
:10402000811109C00E9405240E9462248091E2004F
:1040300084608093E20008958FE398E00E94140565
:104040001092800208958BE398E00E9414050C946E
:104050009D1E87E398E00E94140560917D0281E037
:10406000611101C080E00C94881E83E398E00E94F7
:1040700014059091810281E0943009F080E0609114
:104080007D020C948D1E209143022F5F822F62E3EC
:104090000E942127992319F020934302089510923A
:1040A000430280914702882371F18091810284301C
:1040B00041F58091E9008F702091EC00922F917072
:1040C00020FD90E8892B93E09093E9009091EB001C
:1040D00090FF14C09091EE0097FF10C09091E800FF
:1040E00095FF03C01092F100F9CF9091E80090FF86
:1040F00005C09091E8009E779093E8008F708093C0
:10410000E90010924702089542E061EC81E00E94CC
:104110007E2342E261EC82E00E947E2342E261EC77
:1041200083E00E947E239091810281E0943009F027
:1041300080E060917D020C94961E80918302833012
:1041400009F461C030F4813071F0823009F49AC012
:1041500008958A3009F486C08B3009F46CC0893028
:1041600009F0A8C020C080918202813A09F0A2C063
:104170008091E800877F8093E8008091860290918B
:104180008702892B21F460E288E492E003C060E0BA
:1041900080E090E070E00E94BF228091E8008B7781
:1041A0008093E800089580918202813209F082C0F4
:1041B0008091860290918702029708F07BC08091DF
:1041C000E800877F8093E8008091E80082FD05C0C9
:1041D000809181028111F8CF6DC02091F300809110
:1041E000F20090E0922B029731F48091F10081303F
:1041F00011F0863021F48091F10080936802809163
:10420000E8008B7753C080918202813A09F052C056
:104210008091860290918702892B09F04BC0809192
:10422000E800877F8093E8008091E80080FFFCCF62
:104230008091100136C0809182028132D9F580913F
:10424000860290918702892BA9F58091E800877FEB
:104250008093E8000E94B323809184028093100130
:104260000C94140B80918202813221F58091E80038
:10427000877F8093E8000E94B3238091850280931A
:104280006902089580918202813AA1F48091E80048
:10429000877F8093E8008091E80080FFFCCF8091C9
:1042A00069028093F1008091E8008E778093E800A6
:1042B0000C94B32308959FB7F894109247029FBFC0
:1042C00090918102943009F057C09091E9009F705D
:1042D0003091EC00232F217030FD20E8922B23E059
:1042E0002093E9002091EB0020FF43C02091EE00D5
:1042F00027FF3FC020914202222321F02091E800B5
:1043000025FF37C01092420226E03091E80035FDCB
:1043100015C030918102343061F53091EB0035FDEC
:1043200028C0215021F481E08093420222C0EFE9AD
:10433000FFE03197F1F700C00000E7CF8093F10074
:104340008091E80085FD0AC08091E80080FFFCCFE5
:104350008091E8008E778093E80006C08FB7F894CC
:1043600021E0209347028FBF9F709093E90080E087
:1043700008959F709093E9008FEF089584B7877F29
:1043800084BF0FB6F894A8958091600088618093EF
:104390006000109260000FBE90E080E80FB6F894C5
:1043A00080936100909361000FBE0C94981E0E9450
:1043B00005240E946224E2EEF0E080818460808324
:1043C00078940C94F62684E091E00C94131D80916F
:1043D00081028530C9F48FE298E00E941405809133
:1043E0008102853079F40E94E81E80917F02882343
:1043F000B1F30E94AA1E882391F30E945E220E94BC
:10440000140BEDCF0C94131F089508950C940822FB
:10441000292F332723303105C9F060F421303105CD
:1044200081F02230310509F041C08BE590E02FE5A5
:1044300038E040C021323105E1F02232310531F15E
:1044400035C082E190E02AEB38E034C09927813012
:10445000910549F028F0029749F5E7E4F8E005C036
:10446000EBE5F8E002C0E1E5F8E0849190E09F011F
:1044700021C063307105D0F4660F771FFB01EA5746
:10448000FE4F2081318189E090E014C063307105D6
:1044900068F4FB01EE0FFF1FE058FE4F20813181D1
:1044A000FB01E358FE4F808190E004C080E090E083
:1044B00020E030E0FA0131832083089580E189BD56
:1044C00082E189BD09B400FEFDCF8091D8008F7DC7
:1044D0008093D8008091E00082608093E00080911A
:1044E000E00081FDFCCF0895CF92DF92EF92FF9222
:1044F0000F931F93CF93DF93EC018B017A010E94FE
:10450000D223811133C0E114F10439F0F701808125
:104510009181081B190BC80FD91FC12CD12C011573
:10452000110519F18091E80085FD16C08091E80021
:104530008E778093E800E114F10449F0F70180815F
:104540009181C80ED91ED182C08285E00FC00E9421
:10455000D223882321F30AC089918093F10001506E
:104560001109FFEFCF1ADF0ADACF80E0DF91CF9198
:104570001F910F91FF90EF90DF90CF9008952091C1
:104580008802309189022617370748F061157105B6
:1045900039F42091E8002E772093E80001C0B9019A
:1045A000FC0120E06115710579F180918102882379
:1045B000F1F18530F1F18091E80083FD3CC08091FC
:1045C000E80082FD2EC08091E80080FFEBCF2091B3
:1045D000F3008091F20090E0922B6115710551F08B
:1045E0008830910538F421912093F10061507109D0
:1045F0000196F3CF21E0089709F020E08091E800D0
:104600008E778093E800CECF2111CFCF0AC0809162
:104610008102882361F0853061F08091E80083FD9C
:104620000AC08091E80082FFF2CF80E0089582E026
:10463000089583E0089581E00895209188023091E3
:1046400089022617370748F06115710539F4209162
:10465000E8002E772093E80001C0B901FC0120E0BA
:104660006115710591F180918102882309F440C0A0
:10467000853009F43FC08091E80083FD3DC0809102
:10468000E80082FD2FC08091E80080FFE9CF2091F3
:10469000F3008091F20090E0922B6115710559F0C2
:1046A0008830910540F424912093F10031966150B7
:1046B00071090196F2CF21E0089709F020E080917E
:1046C000E8008E778093E800CBCF2111CCCF0AC0D1
:1046D00080918102882361F0853061F08091E8004B
:1046E00083FD0AC08091E80082FFF2CF80E0089548
:1046F00082E0089583E0089581E00895982F97302F
:1047000068F59093E900981739F07091EC002091CA
:10471000ED005091F00003C0242F762F50E021FDD2
:1047200002C09F5FECCF3091EB003E7F3093EB00F7
:104730003091ED003D7F3093ED003091EB00316022
:104740003093EB007093EC002093ED005093F00059
:104750002091EE0027FDE5CF80E008958F708093D3
:10476000E90081E008958091820287FF11C0809165
:10477000E80082FD05C0809181028111F8CF11C04F
:104780008091E8008B770BC080918102882349F0EB
:104790008091E80080FFF8CF8091E8008E778093C9
:1047A000E80008952091E4003091E50095E64091FD
:1047B000EC00842F817040FF23C08091E80080FDD1
:1047C0001DC080918102882399F0853099F08091F5
:1047D000EB0085FD11C04091E4005091E5002417E5
:1047E000350729F3915011F09A01E1CF84E0089543
:1047F00082E0089583E0089581E0089580E00895BF
:104800004091E80042FFDDCF08950E9473240E948A
:104810007B24E0EEF0E0808181608083E8EDF0E0D1
:1048200080818F77808319BCA7EDB0E08C918E7F5B
:104830008C9380818F7E80831092800208950F93E5
:104840001F93CF93DF930E9473240E947B24C8EDB3
:10485000D0E088818F778883888180688883888189
:104860008F7D888319BC1092810210927D02109274
:104870007F0210927E0200EE10E0F80180818B7FB3
:10488000808388818160888342E060E080E00E94CC
:104890007E23E1EEF0E080818E7F8083E2EEF0E027
:1048A000808181608083808188608083F80180813D
:1048B0008E7F8083888180618883DF91CF911F9173
:1048C0000F910895E8EDF0E080818F7E8083E7ED21
:1048D000F0E080818160808384E082BF81E080930A
:1048E00080020C941F24E8EDF0E080818E7F8083AD
:1048F0001092E20008951092DA001092E1000895FB
:104900001F920F920FB60F9211242F933F934F9344
:104910005F936F937F938F939F93AF93BF93EF9327
:10492000FF938091E10082FF0BC08091E20082FF43
:1049300007C08091E1008B7F8093E1000E944320BB
:104940008091DA0080FF1FC08091D80080FF1BC0DB
:104950008091DA008E7F8093DA008091D90080FF09
:104960000DC080E189BD82E189BD09B400FEFDCFA3
:1049700081E0809381020E940A2005C019BC109238
:1049800081020E941C208091E10080FF19C080916B
:10499000E20080FF15C08091E2008E7F8093E200EC
:1049A0008091E20080618093E2008091D800806273
:1049B0008093D80019BC85E0809381020E94292051
:1049C0008091E10084FF30C08091E20084FF2CC020
:1049D00080E189BD82E189BD09B400FEFDCF8091EF
:1049E000D8008F7D8093D8008091E1008F7E8093E6
:1049F000E1008091E2008F7E8093E2008091E200EE
:104A000081608093E20080917D02882311F084E030
:104A100007C08091E30087FD02C081E001C083E010
:104A2000809381020E9435208091E10083FF29C09C
:104A30008091E20083FF25C08091E100877F809311
:104A4000E10082E08093810210927D028091E1007A
:104A50008E7F8093E1008091E2008E7F8093E20060
:104A60008091E20080618093E20042E060E080E0BB
:104A70000E947E238091F00088608093F0000E9465
:104A80002320FF91EF91BF91AF919F918F917F91E3
:104A90006F915F914F913F912F910F900FBE0F90AB
:104AA0001F9018951F920F920FB60F9211242F93FB
:104AB0003F934F935F936F937F938F939F93AF93A6
:104AC000BF93CF93DF93EF93FF93C091E900CF7033
:104AD0008091EC00D82FD17080FDD0E81092E900D1
:104AE0008091F000877F8093F00078940E94962553
:104AF0001092E9008091F00088608093F000CD2B47
:104B0000CF70C093E900FF91EF91DF91CF91BF91FA
:104B1000AF919F918F917F916F915F914F913F9155
:104B20002F910F900FBE0F901F9018951F93CF934A
:104B3000DF93CDB7DEB7AA970FB6F894DEBF0FBEEE
:104B4000CDBFE2E8F2E08091F100819322E0EA3803
:104B5000F207C9F70E949D208091E80083FF2EC1D3
:104B60008091820290918302492F50E04A30510592
:104B700008F024C1FA01EF55FF4F0C9463278038E9
:104B800021F0823809F01AC108C080917E0290910C
:104B90007F02992389F082600FC0809186028F7016
:104BA000873008F00BC18093E9008091EB0085FB12
:104BB000882780F91092E9009091E800977F909300
:104BC000E8008093F1001092F100D1C0282F2D7FD2
:104BD00009F0F4C0882319F0823061F0EFC08091B1
:104BE0008402813009F0EAC0933009F080E08093BC
:104BF0007F022EC08091840281112AC0809186029A
:104C00008F702FEF280F263008F0D8C08093E9006E
:104C10002091EB0020FF1CC0933021F48091EB0029
:104C2000806214C09091EB0090619093EB0021E0C2
:104C300030E0A90102C0440F551F8A95E2F7409366
:104C4000EA001092EA008091EB0088608093EB000C
:104C50001092E9008091E800877F8093E8000E942D
:104C6000B323ACC08111AAC0109184021F77809138
:104C7000E3008078812B8093E3008091E800877FB8
:104C80008093E8000E94B3238091E80080FFFCCF6E
:104C90008091E30080688093E300111102C082E0FC
:104CA00001C083E08093810289C08058823008F07F
:104CB00085C080918402909185028C3D53E09507D8
:104CC00079F583E08A838AE289834FB7F894DE011D
:104CD000139620E03EE051E2E32FF0E050935700BE
:104CE000E49120FF03C0E295EF703F5FEF708E2FDD
:104CF00090E0EA3010F0C79601C0C0968D939D9366
:104D00002F5F243149F74FBF8091E800877F809360
:104D1000E8006AE270E0CE0101960E94BF2216C050
:104D20006091860270918702AE014F5F5F4F0E94D3
:104D30000622BC01892B09F441C09091E800977FBD
:104D40009093E80089819A810E941D238091E80058
:104D50008B778093E80032C0803881F58091E8003D
:104D6000877F8093E80080917D028093F10080919D
:104D7000E8008E7772CF811121C0809184029091DA
:104D8000850299270297D4F48091E800877F809369
:104D9000E8008091840280937D020E94B323809179
:104DA0007D02811106C08091E30087FD02C081E091
:104DB00001C084E0809381020E9484208091E800F9
:104DC00083FF0AC08091E800877F8093E80080918C
:104DD000EB0080628093EB00AA960FB6F894DEBFDA
:104DE0000FBECDBFDF91CF911F910895CF938091DA
:104DF00081028823A1F0C091E900CF709091EC006E
:104E0000892F817090FD80E8C82B1092E900809175
:104E1000E80083FD0E949625CF70C093E900CF91F2
:104E20000895DB018F939F930E947827BF91AF91E4
:104E3000A29F800D911DA39F900DB29F900D1124F4
:104E40000895991B79E004C0991F961708F0961BE6
:104E5000881F7A95C9F780950895AA1BBB1B51E15D
:104E600007C0AA1FBB1FA617B70710F0A61BB70BDA
:104E7000881F991F5A95A9F780959095BC01CD017F
:104E80000895A1E21A2EAA1BBB1BFD010DC0AA1F8B
:104E9000BB1FEE1FFF1FA217B307E407F50720F0A3
:104EA000A21BB30BE40BF50B661F771F881F991F1E
:104EB0001A9469F760957095809590959B01AC0167
:104EC000BD01CF010895EE0FFF1F0590F491E02D75
:104ED0000994A29FB001B39FC001A39F700D811DD3
:104EE0001124911DB29F700D811D1124911D0895F3
:104EF0000E946927A59F900DB49F900DA49F800DDF
:104F0000911D11240895FB01DC0104C08D910190D5
:104F1000801921F441505040C8F7881B990B08951F
:104F2000F999FECF92BD81BDF89A992780B5089571
:104F3000A8E1B0E042E050E00C94C427262FF99994
:104F4000FECF92BD81BDF89A019700B4021639F0E8
:104F50001FBA20BD0FB6F894FA9AF99A0FBE0895B9
:104F60000396272F0E949F270E949E27252F0E948D
:104F70009F27242F0C949F270196272F0E949F275D
:104F80000C949E27DC01CB01FC01F999FECF06C0F1
:104F9000F2BDE1BDF89A319600B40D9241505040F7
:084FA000B8F70895F894FFCF63
:104FA800C8000102911F951F092005200120941FA8
:104FB80001E200E900EA00B500B600B700CD0083C1
:104FC80001CC008A019201940121022302240225C6
:104FD80002260227022A02B300B4006F0070008183
:104FE8008283E200E900EA00B500B600B700CD0010
:104FF8008301CC008A019201940121022302240238
:105008002502260227022A02B300B4006F007000AE
:10501800818283F1F0C667F7F6F5F49590406D222A
:0C5028005B09EE08CC0871088A08A30898
:00000001FF
